:020000020000FC
:0200000003C03B
:100006005BC002E00EBF0FE50DBF00E00FBB00E1D5
:100016000EBB01E00CBB0DB301BF0DED0EBB01E045
:100026000CBB9DB3977003E007BB08E108BB01EF6B
:1000360000BF0FEF0DBD01E207B911272227B0E07F
:10004600A0E708E101BD0BE001BDC2E7D0E000E496
:1000560009BF7894B49B1EC05E7FB39B29C05D7FA9
:1000660000ED092B06B9B0E0A0E7A89506B104FF9C
:10007600FDCF00000000000000000000000015B1E8
:1000860000ED092B06B920E831E03B172A0711F3EA
:100096001D93ECCFA89550FDDDCF51609A959770D2
:1000A6000DED0EBB9DBB04E00CBB02E00CBBD2CF3A
:1000B600A89593954770D4CF6EE771E06C177D07CE
:0C00C60011F4C2E7D0E089918EBD1895BE
:00000001FF
